:1074000080E189BD82E189BD09B400FEFDCF089508
:10741000AA2069F08091E9008F931092E90090D43E
:1074200083FF01C00FD58F9187708093E900089585
:107430008EEF0090E10008220092E1000895F20131
:10744000F999FECFF2BDE1BD0895F9DFF89A80B554
:1074500008C0F5DF1FBA80BD0FB6F894FA9AF99A02
:107460000FBE31962F0108958BEA3FD0109289000C
:107470008AEF8093880082E080936F0083E080939E
:10748000810098E082E665D0892F877063D08FEF06
:107490005C9860D09A95B2F7E1EAF7E7859159D008
:1074A000E73AE1F781E08093D7008AE482BF109247
:1074B000D8001092E2001092DA001092E10080E809
:1074C00008D019BCAA241092E00050D489E041D41D
:1074D00081E98093D8000895A3E6B1E090E812D046
:1074E0008D939A95E1F7089586E008D017C083E060
:1074F00005D08F2F07D08E2F05D080E05E9A90E5C3
:107500009CBD5A988EBD8DB587FFFDCF8EB5089571
:1075100005D085E0F3DFF6DF80FDFDCF5A9A88E5E0
:107520008CBD5E9808958FE08221E9F7F7DFE3E6EE
:10753000F6E090E080E60DD0892F0CD05C98819128
:1075400009D083E68E278F77D1F79395983091F7FE
:1075500008955C9A5E98D6DF5E9A0895E3E6F1E0BE
:1075600097FC36C094FC4DC092FE089596849920F5
:10757000D1F3F894C089D78520E030E080E090E432
:10758000AFEFBFEF119689199040E0F72D01BD4F85
:107590008D0127FD13C0E0E0F8E011928EE78193A2
:1075A00092E4E11791939AE508F092E4E334C9F785
:1075B00081931082BBDFFE01219699DF8DDFF901F7
:1075C000E3D420583F4F040D151D9A9411F7F8C1CC
:1075D0008301282D60906C0170906B0143D019F4E9
:1075E0008823C1F70895380188243CD0C9F58091DB
:1075F0006A01821709F4830160906E0170906D0139
:10760000F4CF80E1982E60906E0170906D012AD0C9
:1076100059F48823B1F708959FEF95FC03C096FEB7
:10762000089591E097FB890E662477248301222731
:1076300019D0B1F48823A1F380916A0136F088163D
:1076400050F4821730F0213003C0881520F4281739
:1076500010F48301282F60906E0170906D01E8CFC7
:107660003801822EF30143DF37DFC3E6D1E0EAE9D8
:10767000F7E709908591081621F4E13AD1F70880DF
:1076800080104CCFC9E02ADFCA95E9F7D0E197FC1A
:1076900055C094FC37C096FE1AC0C3E6D2E0E3E6BC
:1076A000F6E098E088E78E0F00840192E817E1F792
:1076B000884F09900192E817E1F7C858DF4F9A9573
:1076C00089F731DFC85FD340C33E49F749C0C3E6FD
:1076D000D6E0EBE5FAE098E08E2F8857029000861E
:1076E000E817E1F738960A900292E817E1F7389721
:1076F000C857D0409A9581F716DFC850DC4FC33E7B
:1077000041F72EC0A3EEB6E0E3E6F6E09AE0C6E06D
:107710000D9080818025807F802582958193A3367E
:10772000B90709F4B2E0E336F90709F4F2E0E33609
:10773000FC0771F7F8DEDA9529F712C0A3EEB9E07D
:10774000E3E6FAE092E00E90829180258F7080252A
:1077500082958083E336F907B1F7E5DEDA9571F7B4
:1077600088270895E8EBF0E081818C7F81838CE0AD
:10777000808374E0720D84EA02C0838384E884838A
:10778000848187FD08957211FBCF089502D084E9AA
:10779000848388E08A95F1F7089541524455424F19
:0877A0005924404864008400F4
:1077A8001201100102000008412336000100000008
:1077B800000109023E0002010080320904000001B4
:1077C8000202010005240010010424020405240615
:1077D8000001070582030800FF09040100020A00EE
:1077E80000000705040210000107058302100001CC
:1078000011241FBE04B714BE88E1E0E6F0E08083D7
:1078100011928EEF9AE09EBF8DBF22243324210166
:1078200031014101510187C00F928F939F931F92A5
:107830000FB60F9211244F936F938091DA0080FF5F
:1078400034C020C00F920FB68F939F93EF93FF9396
:1078500088278093850080938400E0E5F1E09081A3
:107860008917980B908309F45D9A91818917980B79
:10787000918309F4289A239411F48315381EFF91FB
:10788000EF9154C08091D80080FF0FC08091DA0042
:107890008E7F8093DA008091D90080FF04C0B0DD34
:1078A00081E0A82E02C019BCAA248091E10080FFCB
:1078B0000BC049D280FF08C049D28091D8008062B5
:1078C00008DE19BC85E0A82E8091E10084FF1AC073
:1078D0003AD284FF17C094DD8091D8008F7DF9DD06
:1078E0008FEEA7DD30D28F7E816033D2809153013D
:1078F000882331F48091E30087FD02C081E001C05C
:1079000084E0A82E8091E10083FF0CC01CD283FF8D
:1079100009C087EF8EDD82E0A82E1092530188DD2A
:1079200015D224D26F914F910F901F909F918F91FC
:107930000FBE0F90189580E880831082B1E0B5BF2C
:1079400082E085BF81EF85B987EE84B91DB8769A4C
:1079500010BA83EF81BB87E78BB984EF8AB980E5E2
:107960008CBDBDBDA0E0E8EAF7E705900D92A0351B
:10797000E1F71D92BB30E9F75F9A04C07C9B02C01F
:107980001FD3F1F471DD78946DDEB0D041DD8FB19D
:107990008095807F66991C9B8460982E3DDE8110C7
:1079A000DDDD882049F492FC09C08FE0822121F4BA
:1079B0008091720187FF18D033203AF701D329F361
:1079C000F89489EB92DD81E08093E00010926F00E3
:1079D00010928100109285001092840085BF15BE20
:1079E0005D9A289A0C940000E5E0F0E080DDA3E6C3
:1079F000B2E0C8E073DDCA95E9F7B4DE80EDBDDE24
:107A000080E0BBDEC3DEB7DE81EDB7DEC4E7D1E0E8
:107A1000DE0184ECB4DE83818D93AA37D1F7AEDE2C
:107A200083818D93B3DE1482AFE2B6E08D8117D0EF
:107A30008C8115D08E8113D09A8190748A8119F02F
:107A40008F7184FF80560BD0898109D0888107D03F
:107A5000992321F08A818695807102D067CD00D06C
:107A60009E01DD91CD91CD59D94FFD91ED91ED590B
:107A7000FE4F41915191549F8295682F6F70609D88
:107A8000E00DF11DBE01152E8E0103561640143077
:107A900050F401900882C058DF4F1A94A9F7EB0107
:107AA00021964A9579F7E901089548D107C009D18F
:107AB00002C0AA2039F044D182FFFBCF85FFF7CF67
:107AC0008091F1000895082E83E039D185FD07C02B
:107AD0002ED102C0AA2049F033D180FFFBCF009203
:107AE000F1005D9884E680935001089527D182FFCC
:107AF000EAC0289884E680935101D7DF182F853497
:107B000031F422248EE7382E9ADC8DE0C5C084350E
:107B100011F4CBDFFACF8C34C1F38035B1F3843765
:107B200011F480E0B9C0813429F4BFDF582EBDDFE5
:107B3000482EEBCF833539F4EAE9F7E78591C3DFC7
:107B4000E13AE1F7AAC0863521F482E3BCDF81E3A4
:107B5000A3C08A3649F48FE9D1DCC3E0D3DCB3DFBC
:107B6000CA95E1F7DBDC99C0833731F487E8ABDFF6
:107B700085E9A9DF8EE190C0823631F489E5A3DF83
:107B800080E0A1DF80E888C0823419F0873609F0F0
:107B90006FC033248ADFD82F88DFC82F86DF082FF5
:107BA0008354843008F077C0063411F4440C551C1B
:107BB000F20110926F001736B9F4033489F483E0B0
:107BC00097DCA0DC8EB51EBC7EDF0DB42197D1F70B
:107BD000A5DC08C0063411F4859101C036DC73DFE2
:107BE0002197C2F72F013CC00334A9F4E11104C06E
:107BF0007BDC88ED7DDC8CDC77DC82E079DC55DFBA
:107C00000DB48EBDCA95D9F731967DDC81DCDA954D
:107C100069F72F0123C00634C1F49F01F437A8F49B
:107C2000C6D113C042DF063461F4C0FB46F0F4371E
:107C300028F4182E81E087BFE89511243296082E8B
:107C400004C0043409F401C004DC21975AF7063457
:107C500029F42F01F901F43708F4A7D18DE033DFBF
:107C6000063411F45694479482E080936F0015C057
:107C70008237E1E049F08634E0E031F08E34E3E031
:107C800019F0813531F4E2E0F0E089E087BF8491BA
:107C900003C08B3111F08FE316DF83E0C6DB47D0E2
:107CA00095FF03C009C0AA2071F04AD080FFFBCF26
:107CB0003ED002C0AA2039F043D080FFFBCF84E041
:107CC000B4DB8BE735C00895E4E5F1E067E090911F
:107CD0005B0180915C01913231F0913A71F5813212
:107CE00061F550D173C0823241F1803231F54AD111
:107CF000AA20E9F08530D9F023D083FD18C082FF97
:107D0000F7CF04C0DDDE8193615031F09091F30034
:107D10008091F200892BB1F7D4DF611549F704C0D7
:107D2000AA2029F0853019F00BD080FFF9CF8EE71B
:107D30009091E80089238093E800089584E075DB42
:107D40008091E80008958091E2000895FCDF8E7F25
:107D500080618093E200089582E061EC09D083E0C5
:107D600061E802D084E060E842E103C080E060E0C6
:107D700042E05BDB81E007D01092ED006093EC0005
:107D80004093ED0008959091EB00892B8093EB00D8
:107D9000089560E0923029F0913029F4E0E062E14A
:107DA00002C0E2E16EE3F1E0089580915B01882377
:107DB0004CF402C0AA20C1F3C3DF82FFFBCF81CF06
:107DC000AA2091F3BDDF80FFFBCFB1CF40916101CD
:107DD000509162014617510520F0462F611509F4B4
:107DE000A6DF50E022C0AA2061F1853051F1A8DF62
:107DF00083FD67CFA5DF82FD21C080FF16C03091D3
:107E0000F3002091F20006C081918093F10041506F
:107E10002F5F3F4F411519F028303105A8F350E08E
:107E20002830310509F451E082DF4115E1F6552390
:107E3000D1F604C0AA2029F0853019F081DF82FF35
:107E4000F9CF3FCFEBE5F1E03BDE8193E336E1F79D
:107E50003BDF76DF83FF91C080915B0190915C01F5
:107E6000913009F170F09330F1F0953009F444C08D
:107E7000963009F456C0983009F460C0993059F72B
:107E800067C0823841F780915F01CEDA2091EB0024
:107E90001092E90077D02295269521702093F10069
:107EA0001092F10052C0882311F08230A1F68F7138
:107EB000823089F680915D018823D1F420915F01A1
:107EC000277049F22093E9008091EB0080FF10C0F9
:107ED000933011F480E20BC080E155DF81E0880F20
:107EE0002A95E9F78093EA001092EA0088E04BDFD8
:107EF0001092E90047D02AC0882391F410915D01C7
:107F000010680FB7F8943ED050DF1ADF80FFFDCF26
:107F10001093E300103883E009F482E0A82E0FBF2D
:107F20002CC08058823048F580915D0190915E01AF
:107F300030DF603011F126D049DF1FC08038E9F40E
:107F400021D0809153018093F100F1DE2EDF15C026
:107F5000882399F490915D01923078F490935301C5
:107F600011D023DF80915301882321F48091E30015
:107F700091E087FD94E0A92EEFDEE2DE83FF089515
:107F800080E201DF87EFD4CEA3E6B1E0F437B8F4A6
:107F90000ED090E40D901D9081E087BFE895329659
:107FA0009A95C1F71124E058F04085E001C083E0C4
:107FB00001D081E187BFE89507B600FCFDCF0895A9
:0C7FC000E0E0F0E08591949101960895B6
:067FFA003231C7CFFBDCB1
:040000030000740085
:00000001FF
